:100000000C945D000C9485000C9485000C94850084
:100010000C9485000C9485000C9485000C9485004C
:100020000C9485000C9485000C9485000C9485003C
:100030000C9485000C9485000C9485000C9485002C
:100040000C94F20C0C9485000C94620D0C943C0DF5
:100050000C9485000C9485000C9485000C9485000C
:100060000C9485000C94850000000008000201003B
:100070000003040700000000000000000000000072
:10008000250028002B0000000000240027002A0083
:10009000040404040404040402020202020203032E
:1000A0000303030301020408102040800102040836
:1000B00010200102040810209C1411241FBECFEF51
:1000C000D8E0DEBFCDBF12E0A0E0B1E0E6E1F1E3B1
:1000D00002C005900D92AC31B107D9F722E0ACE136
:1000E000B2E001C01D92A53DB207E1F710E0CDE5F9
:1000F000D0E004C02197FE010E945D17CC35D107E6
:10010000C9F70E94D2110C9489180C940000FC01CC
:10011000918D228D892F90E0805C9F4F821B9109E9
:100120008F739927089580E090E0892B29F00E9431
:10013000540C81110C9400000895FF920F931F93AB
:10014000CF93DF938B01EA01DB01ED91FC910680F7
:10015000F781E02D60E070E0C8010995F82ED80124
:10016000ED91FC910084F185E02D60E070E0C80124
:100170000995182FE881F9810284F385E02D8F2DF0
:100180000F2C000C990BF7FE09C0AA27BB27A81B50
:10019000B90BA25FBE4F4C91419504C0DC01A25F38
:1001A000BE4F4C9160E070E0CE010995E881F98185
:1001B0000484F585E02D812F012E000C990B17FF8B
:1001C00009C0AA27BB27A81BB90BA25FBE4F4C9141
:1001D000419504C0DC01A25FBE4F4C9160E070E02D
:1001E000CE01DF91CF911F910F91FF900994CF9392
:1001F000DF93FC0198E081E02AB120632AB9282F1F
:1002000030E0220F232F221F330B232B09F427C0AA
:10021000000000000000000000002AB12F7C2AB975
:1002200000000000000000000000000000000000CE
:1002300000000000000000000000000000000000BE
:1002400000000000000000000000000000000000AE
:1002500000000000000000000000000027C00000B7
:10026000000000000000000000000000000000008E
:10027000000000000000000000000000000000007E
:10028000000000000000000000000000000000006E
:10029000000000000000000000000000000000005E
:1002A0000000000000002AB12F7C2AB9915059F0BB
:1002B000000000000000000000000000000000003E
:1002C0000000880F99CF00000000000000008AB1F4
:1002D00080638AB9000000000000000000000000F8
:1002E000000000000000000000000000000000000E
:1002F0008AB18F7C8AB9DF015396AF014D5C5F4FA5
:100300009D018FE399B1907381F08150D9F7128AE2
:10031000118A108A1786D90160E070E0C0E0D0E051
:1003200080E090E040E850E02DC0000000000000B8
:1003300000000000000000000000000000000000BD
:1003400000000000000000000000000000000000AD
:10035000000000000000000000000000000000009D
:1003600000000000000089B180738D934A175B077D
:1003700009F4CDCF8FE399B1907309F0C2CF8150CA
:10038000D1F7C5CF2D91222341F09A01082E02C04A
:10039000359527950A94E2F701C020E0622B179665
:1003A0002C911797222341F09A01082E02C035950F
:1003B00027950A94E2F701C020E0722B1F962C913A
:1003C0001F97222339F09A01082E02C035952795F0
:1003D0000A94E2F7C22B57962C915797222339F0B3
:1003E0009A01082E02C0359527950A94E2F7D22B80
:1003F00001968830910531F6D08BC787728B618B5F
:10040000DF91CF910895DC01ED91FC910284F38599
:10041000E02D6CE070E00994FC012189211104C0F9
:1004200092899F7381E009F080E00895FC012189A1
:10043000211105C092899F7381E09F3309F080E00C
:1004400008959B0177FF02C0295F3F4F43E0359538
:1004500027954A95E1F7FC01E20FF31F218930E06F
:10046000CB0168E070E00E943517A90102C05595E4
:1004700047958A95E2F7CA0181700895FC01808949
:100480000895FC0187850895FC0114A60895FC01D8
:1004900084A50895860F971F4195FC014187089513
:1004A000860F971FFC01418708959B014423E9F0C3
:1004B00077FF02C0295F3F4F53E0359527955A9546
:1004C000E1F7FC01E20FF31FCB0168E070E00E944E
:1004D000351721E030E0A90102C0440F551F8A956D
:1004E000E2F7CA019381892B1DC077FF02C0295F03
:1004F0003F4F43E0359527954A95E1F7FC01E20F20
:10050000F31FCB0168E070E00E94351721E030E076
:10051000A90102C0440F551F8A95E2F7CA018095D0
:100520009381892383830895660F771FFC01E60F6B
:10053000F71F8FE7489F402D1124405846830895A8
:100540006F5F7F4F660F771FFC01E60FF71F8FE786
:10055000489F402D1124405843830895660F771F0C
:10056000860F971F4058FC01468308956F5F7F4FA9
:10057000660F771F860F971F4058FC01438308952D
:10058000FC01138280E88483858386838783808748
:100590001186128608950C94FB1760E070E00C94AD
:1005A0009C10EF92FF920F931F93CF93DF93CDB7E1
:1005B000DEB728970FB6F894DEBF0FBECDBF8C0113
:1005C000FC01E85BFE4F8081833440F4813408F005
:1005D00075C0882331F0803421F187C08F3F09F046
:1005E00084C0FF24F394F0921E0289E0F801838313
:1005F000148283E0858380E88683178210861186C3
:100600001286F386F48640E063E0C80103960E94F8
:10061000E70FF801F4A660E070E0C8010E949C10AA
:1006200064C080911E02882379F0F0901D02F9E0E9
:10063000FF1554F06AE070E080E090E00E949811AD
:10064000F394F0921D0237C010921D0280911C029B
:1006500098012C5D3F4F790181110CC028E0C80141
:100660000396FC01D70101900D922A95E1F741E034
:1006700068E00CC088E0F901DE01119601900D924E
:100680008A95E1F741E068E0CE0101960E94E70F0C
:10069000F801EF2811F4128207C0E65BFE4F80815B
:1006A00081708083F801828361E070E0C8010E945C
:1006B0009C1080931C0210921E0217C010921E0202
:1006C000F801138280E8848385838683878380870B
:1006D0001186128681E08387848741E06AE0C80141
:1006E00003960E94E70F10921D0228960FB6F89409
:1006F000DEBF0FBECDBFDF91CF911F910F91FF9055
:10070000EF900895CF92DF92EF92FF920F931F9395
:10071000CF93DF93EC018B017A018C819D81813035
:10072000910521F0029709F45CC011C0DB01ED9145
:10073000FC910088F189E02DCB010995882329F0EF
:1007400082E090E09D838C836EC11D821C82D70164
:10075000ED91FC91C284D384D801ED91FC91068087
:10076000F781E02D60E070E0C8010995682F880FDF
:10077000770B880B990B0E941316AB01BC01CE01BD
:100780000E94700E482F60E070E0C701F6010995E5
:10079000D701ED91FC91C484D584D801ED91FC91F1
:1007A0000084F185E02D60E070E0C8010995682FB4
:1007B000880F770B880B990B0E941316AB01BC01B5
:1007C000CE010E94700E482F60E070E0C701F60174
:1007D000DF91CF911F910F91FF90EF90DF90CF901D
:1007E0000994DA01ED91FC910284F385E02D4F81AB
:1007F00060E070E0C7010995D701ED91FC91048498
:10080000F585E02D498560E070E0C7010995D801C4
:10081000ED91FC910088F189E02DC80109958823AC
:1008200009F404C18E81D801ED91FC910284F38515
:10083000E02D69E070E0882309F466C0C8010995DD
:1008400081110FC1D801ED91FC910284F385E02D57
:1008500068E070E0C8010995811103C1D801ED91EC
:10086000FC910284F385E02D6BE070E0C8010995EE
:100870008111F7C0D801ED91FC910284F385E02D40
:100880006AE070E0C80109958111EBC0D801ED91D3
:10089000FC910284F385E02D61E070E0C8010995C8
:1008A0008111DFC0D801ED91FC910284F385E02D28
:1008B00060E070E0C80109958111D3C0D801ED91C5
:1008C000FC910284F385E02D62E070E0C801099597
:1008D0008111C7C0D801ED91FC910284F385E02D10
:1008E0006DE070E0C80109958111BBC0D801ED91A0
:1008F000FC910284F385E02D64E070E0C801099565
:100900008111AFC01E82ADC0C8010995882351F086
:100910008F8198858230910514F0019719C081E08C
:1009200090E016C0D801ED91FC910284F385E02D92
:1009300068E070E0C8010995882369F02F81388547
:1009400089859A8501972817390714F4C9010196FA
:1009500098878F8368C0D801ED91FC910284F3855C
:10096000E02D6AE070E0C8010995882361F02985CF
:100970003A858F8198850196821793070CF051C0B4
:10098000C90101974EC0D801ED91FC910284F38515
:10099000E02D6BE070E0C8010995882351F089854E
:1009A0009A858435910514F401963BC08FE390E05D
:1009B00038C0D801ED91FC910284F385E02D64E00C
:1009C00070E0C80109958823D1F08B81813049F00E
:1009D000823071F087E190E098878F8385E290E024
:1009E00020C084E190E098878F8380E290E019C076
:1009F0008EE190E098878F8389E290E012C0D80161
:100A0000ED91FC910284F385E02D6DE070E0C8016A
:100A10000995882331F188E090E098878F838BE1F6
:100A200090E09A87898781E08E831BC08091CD02F8
:100A30009091CE02009799F06F810E94A80A809150
:100A4000CD029091CE02698501960E94A80A8091FC
:100A5000CD029091CE026B8102960E94A80A1D825F
:100A60001C82DF91CF911F910F91FF90EF90DF904B
:100A7000CF900895FC01848DDF01A80FB11DA35A0A
:100A8000BF4F2C91848D90E001968F739927848FAE
:100A9000A689B7892C93A089B1898C9183708064D1
:100AA0008C93938D848D981306C00288F389E02D72
:100AB00080818F7D8083089508950F931F93CF9336
:100AC000DF93EC011A828CE091E0998388831B828A
:100AD0000091CD021091CE0201151105F1F581E0D2
:100AE0000E941F0E8C019093CE028093CD02892B21
:100AF000A1F563E070E081E00E94940D9093CE0236
:100B00008093CD021B8227E130E03E872D8725E2CE
:100B100030E03C872B8727E430E0388B2F8728E0B4
:100B200030E038872F832BE130E03A872987009720
:100B300031F168E00E94A80A8091CD029091CE0226
:100B4000698501960E94A80A8091CD029091CE02FB
:100B50006B8102960E94A80A12C0C8010E94E1148B
:100B600090E098878F83C80101960E94E11490E07D
:100B70009A878987C80102960E94E1148B838B8132
:100B8000813069F08230B1F087E190E09E878D87F7
:100B900085E290E09C878B8787E490E015C084E134
:100BA00090E09E878D8780E290E09C878B8785E32D
:100BB00090E00AC08EE190E09E878D8789E290E008
:100BC0009C878B8789E490E0988B8F8781E090E009
:100BD0009D838C83DF91CF911F910F910895CF92C8
:100BE000DF92EF92FF920F931F93CF93DF93EB016E
:100BF0008A01DA01ED91FC91C088D188E881F98100
:100C00000284F385E02D6BE070E0CE010995F82EAB
:100C1000E881F9810284F385E02D6DE070E0CE017A
:100C200009954F2D481B61E070E0C801F601099558
:100C3000D801ED91FC91E688F788E881F98102847A
:100C4000F385E02D64E070E0CE010995482F64E063
:100C500070E0C801F7010995D801ED91FC91E68893
:100C6000F788E881F9810284F385E02D6AE070E07D
:100C7000CE010995482F6CE070E0C801F701099595
:100C8000D801ED91FC91E688F788E881F98102842A
:100C9000F385E02D69E070E0CE010995482F63E00F
:100CA00070E0C801F7010995D801ED91FC91E68843
:100CB000F788E881F9810284F385E02D68E070E02F
:100CC000CE010995482F62E070E0C801F70109954F
:100CD000D801ED91FC91E688F788E881F9810284DA
:100CE000F385E02D66E070E0CE010995482F61E0C4
:100CF00070E0C801F7010995D801ED91FC91E688F3
:100D0000F788E881F9810284F385E02D67E070E0DF
:100D1000CE010995482F60E070E0C801F701099500
:100D2000D801ED91FC91E688F788E881F981028489
:100D3000F385E02D6CE070E0CE010995482F6DE061
:100D400070E0C801F7010995D801ED91FC91E688A2
:100D5000F788E881F9810284F385E02D65E070E091
:100D6000CE010995482F6EE070E0C801F7010995A2
:100D7000D801ED91FC91E688F788E881F981028439
:100D8000F385E02D63E070E0CE010995482F6BE01C
:100D900070E0C801F7010995D801ED91FC91E68852
:100DA000F788E881F9810284F385E02D62E070E044
:100DB000CE010995482F6AE070E0C801F701099556
:100DC000D801ED91FC91E688F788E881F9810284E9
:100DD000F385E02D61E070E0CE010995482F68E0D1
:100DE00070E0C801F7010995D801ED91FC91E68802
:100DF000F788E881F9810284F385E02D60E070E0F6
:100E0000CE010995482F69E070E0C801F701DF9134
:100E1000CF911F910F91FF90EF90DF90CF900994A9
:100E2000CF92DF92EF92FF920F931F93CF93DF93B6
:100E3000EB018A01DA01ED91FC91C684D784E88147
:100E4000F9810284F385E02D68E070E0CE01099518
:100E5000F82EE881F9810284F385E02D69E070E0E5
:100E6000CE0109954F2D481B61E070E0C801F601E5
:100E70000995D801ED91FC91C088D188E881F9816C
:100E80000284F385E02D6BE070E0CE010995F82E29
:100E9000E881F9810284F385E02D6AE070E0CE01FB
:100EA00009954F2D481B61E070E0C801F6010995D6
:100EB000D801ED91FC91E688F788E881F9810284F8
:100EC000F385E02D64E070E0CE010995482F64E0E1
:100ED00070E0C801F7010995D801ED91FC91E68811
:100EE000F788E881F9810284F385E02D65E070E000
:100EF000CE010995482F6CE070E0C801F701099513
:100F0000D801ED91FC91E688F788E881F9810284A7
:100F1000F385E02D66E070E0CE010995482F61E091
:100F200070E0C801F7010995D801ED91FC91E688C0
:100F3000F788E881F9810284F385E02D67E070E0AD
:100F4000CE010995482F60E070E0C801F7010995CE
:100F5000D801ED91FC91E688F788E881F981028457
:100F6000F385E02D6CE070E0CE010995482F6DE02F
:100F700070E0C801F7010995D801ED91FC91E68870
:100F8000F788E881F9810284F385E02D6DE070E057
:100F9000CE010995482F6EE070E0C801F701099570
:100FA000D801ED91FC91E688F788E881F981028407
:100FB000F385E02D63E070E0CE010995482F6BE0EA
:100FC00070E0C801F7010995D801ED91FC91E68820
:100FD000F788E881F9810284F385E02D62E070E012
:100FE000CE010995482F6AE070E0C801F701099524
:100FF000D801ED91FC91E688F788E881F9810284B7
:10100000F385E02D61E070E0CE010995482F68E09E
:1010100070E0C801F7010995D801ED91FC91E688CF
:10102000F788E881F9810284F385E02D60E070E0C3
:10103000CE010995482F69E070E0C801F701DF9102
:10104000CF911F910F91FF90EF90DF90CF90099477
:10105000CF92DF92EF92FF920F931F93CF93DF9384
:10106000EB018A01DA01ED91FC91C684D784E88115
:10107000F9810284F385E02D68E070E0CE010995E6
:10108000F82EE881F9810284F385E02D69E070E0B3
:10109000CE0109954F2D481B61E070E0C801F601B3
:1010A0000995D801ED91FC91C088D188E881F9813A
:1010B0000284F385E02D6BE070E0CE010995F82EF7
:1010C000E881F9810284F385E02D6AE070E0CE01C9
:1010D00009954F2D481B61E070E0C801F6010995A4
:1010E000D801ED91FC91E688F788E881F9810284C6
:1010F000F385E02D64E070E0CE010995482F64E0AF
:1011000070E0C801F7010995D801ED91FC91E688DE
:10111000F788E881F9810284F385E02D6DE070E0C5
:10112000CE010995482F6CE070E0C801F7010995E0
:10113000D801ED91FC91E688F788E881F981028475
:10114000F385E02D66E070E0CE010995482F61E05F
:1011500070E0C801F7010995D801ED91FC91E6888E
:10116000F788E881F9810284F385E02D67E070E07B
:10117000CE010995482F60E070E0C801F70109959C
:10118000D801ED91FC91E688F788E881F981028425
:10119000F385E02D6CE070E0CE010995482F6DE0FD
:1011A00070E0C801F7010995D801ED91FC91E6883E
:1011B000F788E881F9810284F385E02D65E070E02D
:1011C000CE010995482F6EE070E0C801F70109953E
:1011D000D801ED91FC91E688F788E881F9810284D5
:1011E000F385E02D63E070E0CE010995482F6BE0B8
:1011F00070E0C801F7010995D801ED91FC91E688EE
:10120000F788E881F9810284F385E02D62E070E0DF
:10121000CE010995482F6AE070E0C801F7010995F1
:10122000D801ED91FC91E688F788E881F981028484
:10123000F385E02D61E070E0CE010995482F68E06C
:1012400070E0C801F7010995D801ED91FC91E6889D
:10125000F788E881F9810284F385E02D60E070E091
:10126000CE010995482F69E070E0C801F701DF91D0
:10127000CF911F910F91FF90EF90DF90CF90099445
:101280004F925F926F927F928F929F92AF92BF9296
:10129000CF92DF92EF92FF92CF93DF937B01EA012F
:1012A000DB01ED91FC910680F781E02D60E070E0BC
:1012B000C7010995682F880F770B880B990B0E943F
:1012C00013164B015C01D701ED91FC910084F1856F
:1012D000E02D60E070E0C7010995682F880F770B5B
:1012E000880B990B0E9413166B017C0120E030E003
:1012F0004AEA52E4C501B4010E94691520E030E0D9
:1013000048EC52E40E94C8162B013C0120E030E07A
:10131000A9010E94641587FF11C020E030E04AEA6D
:1013200052E4C501B40190580E94691520E030E0F4
:1013300048EC52E40E94C8162B013C0120E030E04A
:10134000A901C501B4010E94641520E030E0A901A3
:10135000882379F0C501B4010E94641587FD05C09A
:1013600020E030E040E85FE304C020E030E040E807
:101370005FEBC301B2010E94C8164B015C0120E083
:1013800030E04AEA52E4C701B6010E94691520E044
:1013900030E048EC52E40E94C8162B013C0120E0EA
:1013A00030E0A9010E94641587FF11C020E030E001
:1013B0004AEA52E4C701B60190580E94691520E03C
:1013C00030E048EC52E40E94C8162B013C0120E0BA
:1013D00030E0A901C701B6010E94641520E030E0A9
:1013E000A901882379F0C701B6010E94641587FD21
:1013F00005C020E030E040E85FE304C020E030E0DA
:1014000040E85FEBC301B2010E94C8166B017C018A
:1014100020E030E040E053ECC501B4010E946415C7
:1014200087FD11C020E030E040E053E4C501B40185
:101430000E94C31687FD0CC0812C912C3EEFA32E79
:1014400032E4B32E05C0812C912CA12C23ECB22EBA
:1014500020E030E040E053ECC701B6010E94641583
:1014600087FD11C020E030E040E053E4C701B60141
:101470000E94C31687FD0CC0C12CD12C9EEFE92E13
:1014800092E4F92E05C0C12CD12CE12C83ECF82E6E
:10149000C501B4010E94DB15462FE881F981028461
:1014A000F385E02D60E070E0CE010995C701B6013B
:1014B0000E94DB15462FE881F9810484F585E02D33
:1014C00060E070E0CE01DF91CF91FF90EF90DF9070
:1014D000CF90BF90AF909F908F907F906F905F90D4
:1014E0004F900994EF92FF920F931F93CF93DF9346
:1014F0008B01EA01E881F981E284F384DB01ED915B
:10150000FC910680F781E02D60E070E0C80109954C
:10151000482F60E070E0CE01F7010995E881F9817C
:10152000E484F584D801ED91FC910084F185E02DEF
:1015300060E070E0C8010995482F60E070E0CE01DE
:10154000F701DF91CF911F910F91FF90EF900994D8
:101550000F931F93CF938C01C62F0E94E114C817DD
:1015600021F06C2FC8010E94E9148C2FCF911F919C
:101570000F9108952091CF023091D00221153105AD
:1015800029F0682FC90101960C94A80A0895682FC4
:101590008091CF029091D002009711F00C94A80A8C
:1015A00008958091CF029091D002892BF9F480E0C8
:1015B0000E941F0E9093D0028093CF02892BB1F42A
:1015C00062E070E080E00E94940D9093D0028093DE
:1015D000CF02009759F063E00E94A80A8091CF02E1
:1015E0009091D00262E001960C94A80A08950F939E
:1015F0001F93CF93DF938C01EB01FC018381E88182
:10160000F981882359F00684F785E02DCB010995EF
:10161000882309F4E3C0F8011382E0C00284F38553
:10162000E02D64E070E0CE010995882381F083E02D
:1016300090E00E946317FC0112822FEE31E03183AB
:101640002083BC01CE010E94550E80E017C0E881C6
:10165000F9810284F385E02D66E070E0CE01099502
:10166000882391F081E190E00E9463178C010E9431
:101670005D05B801CE010E94550E83E0DF91CF9148
:101680001F910F910C94C70AE881F9810284F385B8
:10169000E02D67E070E0CE010995882381F083E0BA
:1016A00090E00E946317FC01128225EF31E0318344
:1016B0002083BC01CE010E94550E82E0DFCFE8817D
:1016C000F9810284F385E02D6BE070E0CE0109958D
:1016D000882381F083E090E00E946317FC0112826E
:1016E0002BEF31E031832083BC01CE010E94550EE7
:1016F00081E0C4CFE881F9810284F385E02D62E0C6
:1017000070E0CE0109958823D1F082E090E00E943C
:1017100063178C0189EE91E0F801918380838C81BD
:101720009D81009711F00E94FB171D830C838E8111
:101730009F819B838A831F821E8281E049C0E8814A
:10174000F9810284F385E02D60E070E0CE01099517
:101750008823D1F082E090E00E9463178C0183EE31
:1017600091E0F801918380838C819D81009711F035
:101770000E94FB171D830C838E819F819B838A832C
:101780001F821E8282E024C0E881F9810284F385F1
:10179000E02D65E070E0CE0109958823F9F082E044
:1017A00090E00E9463178C018DED91E0F801918328
:1017B00080838C819D81009711F00E94FB171D830F
:1017C0000C838E819F819B838A831F821E8280E08F
:1017D000DF91CF911F910F910C94BA0ADF91CF91B5
:1017E0001F910F910895CF92DF92EF92FF920F9386
:1017F0001F93CF93DF936C017A018B01C0E0D0E09F
:10180000CE15DF0581F0D8016D918D01D601ED91E6
:10181000FC910190F081E02DC6010995892B11F012
:101820002196EECF7E01C701DF91CF911F910F91DD
:10183000FF90EF90DF90CF900895089580E090E0C2
:101840000895FC01538D448D252F30E0842F90E0C6
:10185000821B930B541710F0CF96089501970895AB
:10186000FC01918D828D981761F0828DDF01A80FA8
:10187000B11D5D968C91928D9F5F9F73928F90E0CA
:1018800008958FEF9FEF0895FC01918D828D981739
:1018900031F0828DE80FF11D858D90E008958FEF76
:1018A0009FEF08950E94841880E392E00E948700D1
:1018B00021E0892B09F420E0822F0895EF92FF9216
:1018C0000F931F93CF93DF93EC0181E0888F9B8D63
:1018D0008C8D981305C0E889F989808185FD26C023
:1018E000F62E0B8D10E00F5F1F4F0F731127E02EA8
:1018F0008C8DE8120CC00FB607FCFACFE889F98985
:10190000808185FFF5CFCE010E943A05F1CF8B8D06
:10191000FE01E80FF11DE35AFF4FF0829FB7F894E4
:101920000B8FEA89FB89808180620AC09FB7F89497
:10193000EE89FF896083E889F989808183708064FA
:1019400080839FBF81E090E0DF91CF911F910F9145
:10195000FF90EF900895CF93DF93EC01888D88235B
:10196000C9F0EA89FB89808185FD05C0A889B9890C
:101970008C9186FD0FC00FB607FCF5CF808185FFE7
:10198000F2CFA889B9898C9185FFEDCFCE010E9455
:101990003A05E7CFDF91CF9108953FB7F894809152
:1019A000290290912A02A0912B02B0912C0226B517
:1019B000A89B05C02F3F19F00196A11DB11D3FBF87
:1019C000BA2FA92F982F8827820F911DA11DB11D15
:1019D000BC01CD0142E0660F771F881F991F4A9511
:1019E000D1F708951F920F920FB60F9211242F93E3
:1019F0003F938F939F93AF93BF93809125029091D4
:101A00002602A0912702B09128023091240223E0FF
:101A1000230F2D3720F40196A11DB11D05C026E826
:101A2000230F0296A11DB11D20932402809325024D
:101A300090932602A0932702B09328028091290256
:101A400090912A02A0912B02B0912C020196A11D27
:101A5000B11D8093290290932A02A0932B02B09388
:101A60002C02BF91AF919F918F913F912F910F9039
:101A70000FBE0F901F9018951F920F920FB60F92E6
:101A800011242F933F934F935F936F937F938F9383
:101A90009F93AF93BF93EF93FF9380E392E00E94F5
:101AA0003A05FF91EF91BF91AF919F918F917F91F7
:101AB0006F915F914F913F912F910F900FBE0F90BB
:101AC0001F9018951F920F920FB60F9211242F930B
:101AD0008F939F93EF93FF93E0914002F091410227
:101AE0008081E0914602F091470282FD12C0908110
:101AF000809149028F5F8F7320914A02821751F0C3
:101B0000E0914902F0E0E05DFD4F958F809349023E
:101B100001C08081FF91EF919F918F912F910F9044
:101B20000FBE0F901F9018958F929F92AF92BF9209
:101B3000CF92DF92EF92FF920F931F93CF93DF9399
:101B4000C82E5B01E0902E02F0902F02C0E0D0E0A2
:101B50000AE010E0EC16FD060CF462C0C8010E9419
:101B6000E11498012E5F3F4F49018F3F21F0EC16A1
:101B7000FD0609F04CC0C4010E94E114D82EEC16F9
:101B8000FD0651F090E08A159B050CF440C09C2F97
:101B90008D2FE701E92EF82E6C2DC8010E94A80AAE
:101BA00060E0C80101960E94A80A0D5F1F4FEC1665
:101BB000FD06A1F08D2D90E00297A816B9068CF4D1
:101BC0007801EA0CFB1C6FEFC7010E94A80A6D2D7B
:101BD0006A196350C70102960E94A80A21966A2DCD
:101BE00001C06D2DC4010E94A80A80912E0290911F
:101BF0002F028C179D0749F0D0932F02C0932E021D
:101C00006C2F81E090E00E94A80AC8010BC0C401BB
:101C10000E94E11490E00396080F191F21969ACFB5
:101C200080E090E0DF91CF911F910F91FF90EF90B6
:101C3000DF90CF90BF90AF909F908F900895DF92EC
:101C4000EF92FF920F931F93CF93DF93D82EE090E4
:101C50002E02F0902F0200E010E0CAE0D0E00E1556
:101C60001F05CCF4CE010E94E114D81209C0CE01A8
:101C700001960E94E114811103C0CE0103960DC0AC
:101C8000CE0102960E94E11490E00396C80FD91F7E
:101C90000F5F1F4FE4CF80E090E0DF91CF911F9165
:101CA0000F91FF90EF90DF9008950F931F93CF93C4
:101CB000DF93EC018B018E819F81009721F00E94C0
:101CC000FB171F821E828A819B81009711F00E9460
:101CD000FB171B830A83DF91CF911F910F9108950A
:101CE0002F923F924F925F926F927F928F929F922C
:101CF000AF92BF92CF92DF92EF92FF920F931F931A
:101D0000CF93DF93CDB7DEB728970FB6F894DEBF39
:101D10000FBECDBF9E838D836A017B0120E030E042
:101D200040E053E4C701B6010E94C316181654F4EC
:101D300020E030E040E853E4C701B6010E94F71408
:101D40006B017C0120E030E0A901C701B6010E94CF
:101D5000641587FF0BC0F7FAF094F7F8F094812C24
:101D6000912C90E8A92E9FEBB92E13C020E030E013
:101D7000A901C701B6010E946415882339F0812C9E
:101D8000912C80E8A82E8FE3B82E03C0812C912CD3
:101D90005401ED81FE8127803084B101032C000CB9
:101DA000880B990B0E9413162B013C01A701960189
:101DB0000E946415ED81FE8118160CF4BCC00185EB
:101DC0001285B801012E000C880B990B0E94131686
:101DD00069837A838B839C83A70196010E94C31633
:101DE00018160CF041C0ED81FE810584F685E02DCA
:101DF000FA83E983ED81FE816385748529813A81C7
:101E0000621B730B072E000C880B990B0E94131694
:101E10006D837E838F839887A3019201C701B601EA
:101E20000E94F7149B01AC016D817E818F819885A2
:101E30000E94C8166B017C01B80162197309072E54
:101E4000000C880B990B0E9413169B01AC01C70173
:101E5000B6010E9469156B017C01E981FA81BF011D
:101E6000FF0F880B990B45C020E030E04AEA52E4AE
:101E7000C701B6010E94641587FF42C0ED81FE8153
:101E80000384F485E02DFE83ED8360E470E06E1B37
:101E90007F0B072E000C880B990B0E9413162B0149
:101EA0003C0129813A814B815C81C701B6010E94C6
:101EB000F7149B01AC01C301B2010E94C8166B016B
:101EC0007C0165E570E0601B710B072E000C880B30
:101ED000990B0E9413169B01AC01C701B6010E9429
:101EE00069156B017C012D813E81B901330F880B8F
:101EF000990B0E9413169B01AC01C701B60118C0D3
:101F000020E030E04AEA52E4C701B6010E94F7142B
:101F100020E030E04CE752E40E94C81620E030E0B8
:101F200048E252E40E94691520E030E040E852E4C3
:101F30000E94F81410C065857685072E000C880B6A
:101F4000990B0E941316A70196010E94C816A301BF
:101F500092010E946915A50194010E94C8166B01A7
:101F60007C0120E030E040E053EC0E94641587FDE6
:101F700010C020E030E04EEF52E4C701B6010E94ED
:101F8000C31618164CF0C701B6010E94DB15CB0131
:101F900005C080E89FEF02C08FE790E028960FB65B
:101FA000F894DEBF0FBECDBFDF91CF911F910F918F
:101FB000FF90EF90DF90CF90BF90AF909F908F9069
:101FC0007F906F905F904F903F902F900895FC010D
:101FD00028E0539A808190E0880F892F881F990B01
:101FE000892B09F430C00000000000000000000050
:101FF00000000000000053980000000000000000F6
:1020000000000000000000000000000000000000D0
:1020100000000000000000000000000000000000C0
:1020200000000000000000000000000000000000B0
:1020300000000000000000000000000000000000A0
:102040000000000030C000000000000000000000A0
:102050000000000000000000000000000000000080
:102060000000000000000000000000000000000070
:102070000000000000000000000000000000000060
:102080000000000000000000000000000000000050
:102090000000000000000000000000000000000040
:1020A000000000005398215069F00000000000007B
:1020B0000000000000000000000000008081880F88
:1020C000808387CF0000000000000000615031F0E5
:1020D000000000000000000031967ACF00000000F0
:1020E000000000000000000000000000539A000003
:1020F00000000000000000000000000000000000E0
:10210000000000000000000000000000442391F0E7
:1021100000000000000000000000000000000000BF
:1021200000000000000000000000000000000000AF
:102130000000000053980895CF93DF93DC01FC0169
:10214000E85BFE4F83E0EF0119928A95E9F7EF0112
:10215000161617069CF484EC99E04B9907C081E0B1
:102160009C968C939C9728E030E01BC00197A9F7C0
:102170009C968C919C97882309F461C09C968C91C5
:102180009C9781110AC080E290E04B9902C080E2E6
:1021900090E0019718161906C4F328E030E04B9937
:1021A000FECF000000000000000000000000000062
:1021B000000000000000000000000000000000001F
:1021C000000000000000000000000000000000000F
:1021D00000000000000000000000000000000000FF
:1021E00000000000000000000000000000004B9B09
:1021F00003C08081816080832150310931F080816A
:10220000880F80834B9BFECFCACF8881803441F4F6
:10221000CD01865B9E4FE817F90711F03196BDCFCF
:102220004B9BFECF8CE090E04B9902C08CE090E09D
:10223000019718161906C4F381E090E002C080E00F
:1022400090E0DF91CF910895CF93DF9390E0FC0170
:10225000EC55FF4F2491FC01E057FF4F84918823F8
:10226000C1F090E0880F991FFC01EA57FF4FC5911C
:10227000D491FC01E458FF4FA591B4919FB7F89415
:102280008881E22FE0958E2388838C91E823EC935C
:102290009FBFDF91CF91089590E0FC01E859FF4F77
:1022A0002491FC01EC55FF4F3491FC01E057FF4FA6
:1022B000E491EE23B9F1222339F1233091F038F47F
:1022C0002130A9F0223001F584B58F7D12C027306E
:1022D00091F02830A1F02430B9F4809180008F7DF6
:1022E00003C0809180008F77809380000DC084B5FB
:1022F0008F7784BD09C08091B0008F7703C0809133
:10230000B0008F7D8093B000F0E0EE0FFF1FE45827
:10231000FF4FA591B4919FB7F8948C9130953823D5
:102320003C939FBF0895682F80E392E00C945E0C6D
:102330008F929F92AF92BF92CF92DF92EF92FF92D5
:102340006B017C010E94CD0C4B015C01C114D104D6
:10235000E104F104F1F00E94CD0CDC01CB018819FD
:102360009909AA09BB09883E9340A105B10570F3FC
:1023700021E0C21AD108E108F10888EE880E83E056
:10238000981EA11CB11CC114D104E104F10419F779
:10239000DDCFFF90EF90DF90CF90BF90AF909F90F8
:1023A0008F900895CF93DF9300D01F92CDB7DEB703
:1023B000789484B5826084BD84B5816084BD85B520
:1023C000826085BD85B5816085BD80916E0081602C
:1023D00080936E00109281008091810082608093D2
:1023E00081008091810081608093810080918000D4
:1023F0008160809380008091B10084608093B100FF
:102400008091B00081608093B00080917A008460F8
:1024100080937A0080917A00826080937A00809124
:102420007A00816080937A0080917A00806880933E
:102430007A001092C100E0914002F091410282E0E6
:102440008083E0913C02F0913D021082E0913E02D7
:10245000F0913F0280E1808310924802E0914402B3
:10246000F091450286E08083E0914202F0914302C0
:10247000808180618083E0914202F09143028081FB
:1024800088608083E0914202F091430280818068FD
:102490008083E0914202F091430280818F7D8083AE
:1024A0008091000190910101019790930101809327
:1024B000000143E050E062E070E0CE0101960E942E
:1024C000D1148981853A31F48A818E3919F48B814E
:1024D0008C3811F080E04DC089E090E00E94E1145A
:1024E0008233A1F162E389E090E00E94A80A109291
:1024F0002F0210922E0260E080E090E00E94A80A75
:1025000060912E0281E090E00E94A80A80918E01E5
:1025100090918F01A091900189839A83AB83CE0122
:1025200001967C0102E010E0D701DD907D01C80139
:102530000E94E114D81621F06D2DC8010E94E91403
:102540000F5F1F4F0530110579F712C080E090E052
:102550000E94E11490E090932F0280932E0281E07C
:1025600090E00E94E11490E090932F0280932E025D
:1025700081E0809323028BE491E00E9463178C0139
:1025800085E991E0F80191838083339651E2F52E3D
:10259000DF018F2D1D928A95E9F7EB5BFE4F83E0FB
:1025A000DF011D928A95E9F7F80114A61093220223
:1025B0000093210284E390E00E946317FC0187EC02
:1025C00091E0918380831786108A118A128ACF0145
:1025D0004396DC011D92FA94E9F79587848780E29F
:1025E00090E0938782871686F0932002E0931F0283
:1025F00083E00E944C1183E00E942411F8011282B2
:102600000E94D10A8091CF029091D0020097C1F030
:1026100001960E94E114813049F0823089F082E015
:1026200090E00E9463172DED31E010C082E090E051
:102630000E94631729EE31E0FC013183208309C039
:1026400082E090E00E94631723EE31E0DC012D93DD
:102650003C936C010E94D10A8091CF029091D002EC
:102660000097F9F00E94E1148230D9F0833021F113
:10267000813049F083E090E00E946317FC011282F0
:102680002FEE31E016C083E090E00E946317DC017A
:1026900012961C9212972BEF31E02D933C938C01F4
:1026A00012C083E090E00E946317FC01128225EFC4
:1026B00031E031832083F3CF81E190E00E94631702
:1026C0008C010E945D05A0902102B0902202E09052
:1026D0001F02F090200285E00E944C1185E00E94CC
:1026E000241184E00E944C1184E00E942411D7013F
:1026F0001996BC92AE92189712960C931297139655
:102700001C9313971496CC9214971596DC921597F8
:1027100017961C921E92169731E0632E32E0732EAC
:102720005524539448E0842E912C809123028823D1
:1027300009F4F7C08091210290912202DC01ED9111
:10274000FC910190F081E02D09958111D2C000919A
:102750001F0210912002F8018685C484D584A284CA
:10276000B384882351F1E12CF12CEA14FB0464F5C5
:10277000C701F7FC079623E0959587952A95E1F721
:10278000F601E80FF91F2081022E000C330BC70160
:10279000B4010E94351702C0359527958A95E2F756
:1027A000C9018170992720FF02C081E390E00E9457
:1027B0009311FFEFEF1AFF0AD8CF7601C7018C19EA
:1027C0009D098A159B057CF08AE090E00E94931198
:1027D000D801ED91FC910484F585E02DC80109959F
:1027E00081110EC038C0F70181917F01882319F053
:1027F00081E390E002C080E090E00E949311DECF80
:10280000D8011296ED91FC911397309719F08281BF
:10281000811121C084E090E00E9463177C01FC01DB
:102820007182608253825282892B09F47DC0F80143
:1028300086819781009711F00E94FB17D8011296AC
:102840008D919C91139717969C938E931697139640
:10285000FC92EE9212976091000170910101072E97
:10286000000C880B990B0E949811F89400911F029C
:1028700010912002D801ED91FC910480F581E02DAA
:10288000C8010995F80180859185DC01ED91FC91E5
:102890000084F185E02D0995F801828193810097EC
:1028A00051F040855185DC01ED91FC910190F08162
:1028B000E02DB8010995F80186819781892B71F483
:1028C00084819581009751F040855185DC01ED911F
:1028D000FC910190F081E02DB801099580912102D1
:1028E00090912202DC01ED91FC910480F581E02DB4
:1028F00009958091210290912202DC01ED91FC91D9
:102900000280F381E02D0995F89480912102909145
:102910002202DC01ED91FC910680F781E02D099502
:1029200078940E94930001CFF80186819781938368
:102930008283178216828FCFE0E3F2E01382128245
:1029400088EE93E0A0E0B0E084839583A683B7830C
:102950008DE092E09183808385EC90E09587848779
:1029600084EC90E09787868780EC90E0918B808B59
:1029700081EC90E0938B828B82EC90E0958B848B42
:1029800086EC90E0978B868B118E128E138E148EB0
:102990001092CE021092CD021092D0021092CF026D
:1029A0000895DC01CB01FC01F999FECF06C0F2BD10
:1029B000E1BDF89A319600B40D9241505040B8F7FD
:1029C0000895F999FECF92BD81BDF89A992780B5F7
:1029D0000895262FF999FECF1FBA92BD81BD20BD63
:1029E0000FB6F894FA9AF99A0FBE019608955058C6
:1029F000BB27AA270E940F150C9489160E947B16EC
:102A000038F00E94821620F039F49F3F19F426F422
:102A10000C9478160EF4E095E7FB0C947216E92FEF
:102A20000E949A1658F3BA1762077307840795072E
:102A300020F079F4A6F50C94BC160EF4E0950B2E5C
:102A4000BA2FA02D0B01B90190010C01CA01A00100
:102A50001124FF27591B99F0593F50F4503E68F15B
:102A60001A16F040A22F232F342F4427585FF3CF9C
:102A7000469537952795A795F0405395C9F77EF46D
:102A80001F16BA0B620B730B840BBAF09150A1F0B6
:102A9000FF0FBB1F661F771F881FC2F70EC0BA0F3C
:102AA000621F731F841F48F4879577956795B795C4
:102AB000F7959E3F08F0B0CF9395880F08F09927BF
:102AC000EE0F9795879508950E944E1608F481E0C1
:102AD00008950E947D150C9489160E94821658F064
:102AE0000E947B1640F029F45F3F29F00C94721687
:102AF00051110C94BD160C9478160E949A1668F326
:102B00009923B1F3552391F3951B550BBB27AA27A6
:102B100062177307840738F09F5F5F4F220F331FE0
:102B2000441FAA1FA9F335D00E2E3AF0E0E832D0A8
:102B300091505040E695001CCAF72BD0FE2F29D0AB
:102B4000660F771F881FBB1F261737074807AB077D
:102B5000B0E809F0BB0B802DBF01FF2793585F4FF2
:102B60003AF09E3F510578F00C9472160C94BD1605
:102B70005F3FE4F3983ED4F3869577956795B795D4
:102B8000F7959F5FC9F7880F911D9695879597F9DF
:102B90000895E1E0660F771F881FBB1F6217730758
:102BA0008407BA0720F0621B730B840BBA0BEE1F6D
:102BB00088F7E09508950E94E2156894B1110C948D
:102BC000BD1608950E94A21688F09F5798F0B92F5D
:102BD0009927B751B0F0E1F0660F771F881F991F52
:102BE0001AF0BA95C9F714C0B13091F00E94BC1622
:102BF000B1E008950C94BC16672F782F8827B85F32
:102C000039F0B93FCCF3869577956795B395D9F7A9
:102C10003EF490958095709561957F4F8F4F9F4FB3
:102C20000895E89409C097FB3EF4909580957095BF
:102C300061957F4F8F4F9F4F9923A9F0F92F96E908
:102C4000BB279395F695879577956795B795F1117D
:102C5000F8CFFAF4BB0F11F460FF1BC06F5F7F4F1A
:102C60008F4F9F4F16C0882311F096E911C077232C
:102C700021F09EE8872F762F05C0662371F096E835
:102C8000862F70E060E02AF09A95660F771F881F04
:102C9000DAF7880F9695879597F90895990F0008A8
:102CA000550FAA0BE0E8FEEF16161706E807F9071E
:102CB000C0F012161306E407F50798F0621B730BB9
:102CC000840B950B39F40A2661F0232B242B252B3A
:102CD00021F408950A2609F4A140A6958FEF811DDD
:102CE000811D089597F99F6780E870E060E008957E
:102CF0009FEF80EC089500240A9416161706180614
:102D00000906089500240A941216130614060506EF
:102D10000895092E0394000C11F4882352F0BB0F80
:102D200040F4BF2B11F460FF04C06F5F7F4F8F4FE3
:102D30009F4F089557FD9058440F551F59F05F3F1E
:102D400071F04795880F97FB991F61F09F3F79F0CD
:102D500087950895121613061406551FF2CF46954F
:102D6000F1DF08C0161617061806991FF1CF8695D1
:102D70007105610508940895E894BB2766277727B5
:102D8000CB0197F908950E944E1608F48FEF08952D
:102D90000E94DB160C9489160E947B1638F00E9464
:102DA000821620F0952311F00C9472160C9478166C
:102DB00011240C94BD160E949A1670F3959FC1F3CE
:102DC000950F50E0551F629FF001729FBB27F00DD9
:102DD000B11D639FAA27F00DB11DAA1F649F66272E
:102DE000B00DA11D661F829F2227B00DA11D621F7D
:102DF000739FB00DA11D621F839FA00D611D221F37
:102E0000749F3327A00D611D231F849F600D211D1A
:102E1000822F762F6A2F11249F5750409AF0F1F09D
:102E200088234AF0EE0FFF1FBB1F661F771F881F06
:102E300091505040A9F79E3F510580F00C947216B6
:102E40000C94BD165F3FE4F3983ED4F386957795D6
:102E50006795B795F795E7959F5FC1F7FE2B880FAC
:102E6000911D9695879597F9089597FB072E16F46F
:102E7000009407D077FD09D00E94491707FC05D0C0
:102E80003EF4909581959F4F0895709561957F4F81
:102E90000895AA1BBB1B51E107C0AA1FBB1FA617A1
:102EA000B70710F0A61BB70B881F991F5A95A9F7F3
:102EB00080959095BC01CD010895EE0FFF1F059000
:102EC000F491E02D09940F931F93CF93DF938230F9
:102ED000910510F482E090E0E091D302F091D402E9
:102EE00020E030E0A0E0B0E0309719F1408151815E
:102EF0000281138148175907C8F08417950769F4B0
:102F0000109731F012960C93129713961C9327C0CA
:102F10000093D3021093D40222C02115310519F079
:102F20004217530718F49A01BD01EF01DF01F801C0
:102F3000DBCF21153105F9F0281B390B2430310581
:102F400080F48A819B816115710521F0FB019383D7
:102F5000828304C09093D4028093D302FE01329600
:102F600044C0FE01E20FF31F819391932250310977
:102F7000398328833AC02091D1023091D202232B89
:102F800041F420910401309105013093D202209345
:102F9000D10220910201309103012115310541F444
:102FA0002DB73EB74091060150910701241B350B08
:102FB000E091D102F091D202E217F307A0F42E1BA8
:102FC0003F0B2817390778F0AC014E5F5F4F24178D
:102FD000350748F04E0F5F1F5093D2024093D10245
:102FE0008193919302C0E0E0F0E0CF01DF91CF91B7
:102FF0001F910F910895CF93DF93009709F481C03B
:10300000FC01329713821282A091D302B091D402B4
:10301000109781F420813181820F931F2091D1027A
:103020003091D2022817390751F5F093D202E0937C
:10303000D10267C0ED0120E030E0CE17DF0740F499
:103040004A815B819E0141155105F1F0EA01F5CFFE
:10305000D383C28340815181840F951FC817D9073C
:1030600059F488819981840F951F029691838083FA
:103070008A819B81938382832115310529F4F09302
:10308000D402E093D3023DC0E901FB83EA83499176
:103090005991C40FD51FEC17FD0761F48081918110
:1030A000840F951F0296E901998388838281938119
:1030B0009B838A83E0E0F0E012968D919C911397B8
:1030C000009719F0FD01DC01F7CF8D919C911197CC
:1030D0009D012E5F3F4F820F931F2091D1023091AF
:1030E000D2022817390769F4309729F41092D402D4
:1030F0001092D30202C013821282B093D202A09324
:10310000D102DF91CF91089581E090E0F8940C9482
:063110008918F894FFCFBE
:103116000C000000D50280000000000082030010B1
:10312600111213141516171718191A1B1B1C1D1E1E
:103136001E1F20212222232424252626272828294B
:103146002A2A2B2C2C2D2D2E2F2F30303131323395
:1031560033343435353636373738383839393A3AFC
:103166003B3B3B3C3C3D3D3D3E3E3F3F3F40404080
:103176004041414142424243434343434444444421
:1031860044454545454546464646464646464646E0
:103196004747474747474747474747474747A59E04
:1031A6008C0000000047024402CD02D102C002B6E4
:1031B60002AE02A002940250024A0255020000002A
:1031C6000000000000520C520C520C520C520C52D1
:1031D6000C520C000000005C05CB02F70041023ED9
:1031E60002210216020C0203020000000010070072
:1031F600000000EF05000000002808000000007233
:103206000A000000009D00000000004009000000C8
:1032160000F70A00000000520C000000005E0CF3EC
:0C3226000B210CAB0C8700300C440C009A
:00000001FF
